:10000000F8FF022099010000911700004917000035
:100010004917000049170000491700004917000060
:100020004917000049170000491700009117000008
:1000300091170000491700003D1F000041200000FB
:100040009117000091170000911700009117000010
:100050009117000091170000911700009117000000
:1000600091170000911700009117000091170000F0
:1000700091170000911700009117000091170000E0
:1000800091170000911700009117000091170000D0
:1000900091170000911700009117000091170000C0
:1000A00091170000911700009117000091170000B0
:1000B000911700009117000091170000C917000068
:1000C00091170000F518000091170000211A000098
:1000D00091170000191B00009117000091170000F4
:1000E0009117000091170000911700009117000070
:1000F0009117000091170000911700009117000060
:10010000911700009117000091170000911700004F
:1001100091170000E90800009117000091170000F6
:10012000911700009117000091170000911700002F
:10013000911700009117000091170000911700001F
:100140009117000091170000111C0000911700008A
:10015000091D000091170000911700009117000081
:1001600091170000911700009117000091170000EF
:1001700091170000911700009117000091170000DF
:1001800091170000911700009117000091170000CF
:100190009117000091170000584B4CF2205210B5F7
:1001A0001A804DF628121A8000BF00BF01F0F4FA41
:1001B000534B4FF030621A60524A9A60524ADA60EA
:1001C000524B4FF470021A60514A136813F4807353
:1001D00004D150490B604FF4A85313604E4B1A786A
:1001E000110703D51A7842F008021A704B4B4C499C
:1001F0002A221A704B4A4C4B8B4204D252F8040FFD
:1002000043F8040BF8E7494B494900228B4202D2DC
:1002100043F8042BFAE74749474A002352F82300E2
:1002200041F823000133662BF8D1444B444A802126
:1002300003F8011B9342FBD1424B3E4A1A60424BEA
:100240008A221A70A3F5805324225A70A0221A70B1
:100250009A799207FCD59A79D406FCD43B4A9379D3
:1002600003F00C03082B394BF9D103221A714022F9
:100270005A719A799006FCD5344A9179334B4906E4
:10028000FBD5334A334911600221516020221A7094
:100290009A7902F00C020C2AFAD12F4B2F4A1A60DD
:1002A0002F4B4BF67F321A6000225A60072243F828
:1002B000042C2C4AC3F80C2D62B600F0BDF9154B86
:1002C0001B68DA0705D5284800F04AF9274B284A69
:1002D0001A60284B1B785B0609D5244C244B2268F6
:1002E0009A4204D1204800F03BF90023236001F03A
:1002F000E3FE01F057FA01F04DF9FEE70E2005404C
:1003000030800440823F04000100002B88ED00E0B3
:1003100010D0034014D0034002D0074000E0074053
:10032000280CFF1F94240000F806FF1F280CFF1F55
:100330006410FF1F0002FF1F0000000000E400E047
:1003400056E400E008ED00E00050064000400640A2
:10035000448004400000131104800440C0100500D4
:1003600014E000E000002020ADC39A5D1CE00340D3
:10037000A5C3945A00F00740FFFFFFFFFFFFFFFFF8
:10038000FFFFFFFFFFFFFFFFFFFFFFFFFFFFFFFF7D
:10039000FFFFFFFFFFFFFFFFFFFFFFFFFFFFFFFF6D
:1003A000FFFFFFFFFFFFFFFFFFFFFFFFFFFFFFFF5D
:1003B000FFFFFFFFFFFFFFFFFFFFFFFFFFFFFFFF4D
:1003C000FFFFFFFFFFFFFFFFFFFFFFFFFFFFFFFF3D
:1003D000FFFFFFFFFFFFFFFFFFFFFFFFFFFFFFFF2D
:1003E000FFFFFFFFFFFFFFFFFFFFFFFFFFFFFFFF1D
:1003F000FFFFFFFFFFFFFFFFFFFFFFFFFFFFFFFF0D
:10040000FFFFFFFFFFFFFFFFFFFFFFFFDEF9FFFF23
:1004100010B5054C237833B9044B13B10448AFF33E
:1004200000800123237010BD280CFF1F0000000076
:1004300098240000084B10B51BB108490848AFF3D9
:1004400000800848036803B910BD074B002BFBD0A0
:10045000BDE81040184700BF000000002C0CFF1F33
:1004600098240000280CFF1F0000000001210D202F
:1004700000F08EB808B501210D2000F083F84FF48C
:100480007A7000F08BF80D20002100F07BF84FF41B
:100490007A70BDE8084000F081B800BF10B4114B7D
:1004A00053F8302092F8804234B1012379B182F8B8
:1004B00080305DF8044B704703EBC0035B681A683B
:1004C00051B922F002021A605DF8044B704782F8BD
:1004D00000315DF8044B704742F003021A605DF88A
:1004E000044B7047F42100001C4A02EBC0030129B1
:1004F0005B6811D004291BD052F83000002280F82C
:10050000802229B1022920D0032922D01A60704705
:100510004FF480721A60704752F830004FF4A272A4
:1005200080F880121A601A6822F020021A60704760
:1005300052F830104FF4A272012081F880021A6044
:100540001A6842F020021A60704740F203121A60E3
:1005500070474FF481721A60704700BFF4210000A9
:1005600030B4054B054D064C002210211A602A605C
:100570002060196030BC704714D0034004D00340A1
:1005800000D003403F2801D8FFF788BF704700BF65
:100590003F2801D8FFF7A8BF704700BF2DE9F843F7
:1005A000054672B6204F214B214A1B683C681268F1
:1005B00062B6520102D5322B88BF013495B3C3F520
:1005C0003B431C4EDFF86490DFF864807F334FF4C8
:1005D0007A72A6FB031302FB04F404EB531472B605
:1005E000D9F800103A68D8F800E062B6C1F53B438C
:1005F0007F33A6FB03031EF0806FC4EB53134FF44D
:100600007A7002D0322988BF013200FB0233B3F581
:100610007A7F04D3013D05D004F57A74DFE700F05A
:10062000C1FFDCE7BDE8F883440CFF1F18E000E0E1
:1006300004ED00E0ABAAAAAAF8B53E4B3E49DFF8AC
:1006400018C13E4E3E4ADFF814E13E4D3E4C3F4F4E
:100650004FF0006018604FF0805018604FF000506D
:1006600018604FF0804018604FF000401860002084
:10067000086028234BF6FF71CCF80010CEF800304C
:1006800033600EF5012E13602B60236005F5002505
:100690003B6004F50024B36207F50027936206F57A
:1006A000012602F501220EF1100E05F6E87504F69A
:1006B000E87407F57F67103220362B602360CEF890
:1006C00000303B6013603360214EBB6193610922AF
:1006D0003260A7F5002706F58056203F08363860BF
:1006E0003160BB60F36047F8042C06F5FD2607F582
:1006F000FE2706F2FC76043730603960B360FB6099
:1007000046F8042C0836C7F8FC0F06F6FC761148AC
:1007100031602B602360026000F0A6FF1920FFF714
:100720003DFF00F025FE40F21310BDE8F840FFF752
:1007300035BF00BF04E100E00480034014800340A3
:100740001C800340248003402C80034034800340FD
:100750000080034000900B40088003400C80034061
:10076000431E032B14D872B60A4951F8230068B10E
:1007700070B4094C058834F81320466841F82360AA
:10078000521B24F8132062B670BC704762B67047E3
:1007900000207047A00CFF1F5C10FF1F30B472B622
:1007A0002B4A13781D0706D52A4B196A002936D023
:1007B000996A002941D053781C0706D5254B196C3E
:1007C00000293ED0996C002939D09378190705D5B6
:1007D000204B196E002936D0996E89B1D3781B074A
:1007E00007D51C4BD3F880207AB3D3F88820112189
:1007F0003AB162B6184B00221A7030BC00F052BEFB
:100800000D21154C154D227843F8315003EBC103EF
:100810000830013A5860227062B630BC704704223A
:100820000D4C0F4D217843F8325003EBC2030830D2
:100830004A1E5860227062B6EFE70521E1E7092100
:10084000DFE70822ECE70C22EAE71022E8E700BF26
:10085000F42300000000FF1F1D0DFF1FC800400013
:1008600088004000431E032B1DD81B4A400140F066
:10087000100030B4104472B6184CE25C032A1BD846
:10088000DFE802F00212151703220D88E25410F07F
:10089000080F14BFC823882343EA054308310360C7
:1008A000416062B630BC704708300222EDE7052295
:1008B000EBE708300422E8E7094A52F8230038B190
:1008C000084A52F82300416042F8231062B6E9E773
:1008D00042F82310034AF7E70000FF1F2C0DFF1F0B
:1008E000F40CFF1F040DFF1F2DE9F04FDFF814B3C8
:1008F000DFF814A387B044E0AC4F4FEA930807EB4E
:10090000C809013ED9F8042003F00803F6B2A2F1A9
:10091000080003F0FF04002B40F0FF8057F8383048
:100920001B0C99B222F8081C002B00F0ED80A04BA4
:1009300022F8064C42F8044C53F82620002A00F016
:10094000CD819C4D55F8263058609B4C45F82600CB
:1009500034F81630194424F8161000F083FD0028EE
:1009600000F0C081954A964B19F0080F00F108007D
:1009700018BF1346C9F8040047F8383008238BF82D
:1009800000309BF80040E4B265071AD58D4B1B7808
:10099000A3B18D490A7802F0FF0322B1013BDBB21B
:1009A0000B7003B900BE89490A7802F0FF032AB12F
:1009B000013BDBB20B70002B00F0668104238BF847
:1009C000003004F0080303F0FF02002B00F0C980A0
:1009D0009AF80030DBB21E098ED19A08DFF8CC916C
:1009E00059F8321009EBC200C1F3830101394068A4
:1009F0000C2900F28580DFE801F07A7A8383838313
:100A000083834683838307000168714D4068714F7B
:100A1000714E6860296088B240F281610024674BA2
:100A200049F832304FF0010E88423C60C9F810405E
:100A3000C9F8184086F800E05C4A00F2E780B0F59B
:100A4000D06F80F01B82B0F5817F00F0D98100F279
:100A50006981802800F02A82822840F0D781A98805
:100A600001F07F01042900F2D1815C485C4A8900D1
:100A700008441470547001788C0740F1608382F848
:100A800000E0022173E1534F3A682AB3554B524EAE
:100A9000554819883478057840298E4645F0020873
:100AA00028BF4FF0400E002C84F001043470CEEBD0
:100AB00001010CBF8824C82409EBC80689B285F05F
:100AC000010544EA0E447260198049F838407244C6
:100AD0000570002965D03A603D4B1A88B2F5A06FC9
:100AE0000ED100219A785970404B1A7008E03849AD
:100AF0003F4C0D68A54200F09880304949F832100B
:100B00003C4A0123137039E72C4A2D4B19F0080F8A
:100B100018BF134647F8383030E700F0C3FC364AB8
:100B2000364952F82630002B00F0E38058688C5D7F
:100B300042F8260003F10802C9F80420032C05D866
:100B4000DFE804F02C02292602228A551A8819F0BF
:100B5000080F0CBF8823C82343EA024347F8383004
:100B60000CE7E00700F19380210600F1D180A20795
:100B700006D5234A234913780220DBB2137008708C
:100B8000E30602D51F4B10221A7007B0BDE8F08FA4
:100B900004228A55DAE705228A55D7E703228A55C7
:100BA000D4E7BEF1400F18BF002294E70000FF1FFA
:100BB000A00CFF1F4C0CFF1F5C10FF1FC800400063
:100BC00088004000280DFF1FB10CFF1F3C0DFF1FC8
:100BD000140DFF1F480CFF1FB00CFF1FC020074063
:100BE000200DFF1F5C0CFF1F1C0DFF1F98200740EE
:100BF0002109000394200740F40CFF1F2C0DFF1F58
:100C0000882007408020074090200740B0F5106FF3
:100C100000F07C8140F2A38040F62112904240F027
:100C20007B82A54A012313706AE74C68A3498C4272
:100C30007FF463AF0178A9297FF45FAF417845293C
:100C40007FF45BAF8178C2297FF457AFC1786B29FD
:100C50007FF453AF9A489B4E0178347881F00105B8
:100C6000002C41F0020105700CBF8820C82084F0E0
:100C7000010449F8310009EBC101934834700025A3
:100C800005244D60047038E700F064FC96E68F4B55
:100C900089488B491A614FF0020E80F800E08C4FB2
:100CA0000A708C49196099608B4E8C4D8C4C9A61FE
:100CB0000D213970FF213170DFF84CE2297022706C
:100CC000884D894A8EF800109F27012406F8047C7D
:100CD0005D600470DA6007B0BDE8F08F43F826006D
:100CE000824D32E6824A47F8380013780133137098
:100CF00044E68B5D032B00F2BA8001A252F823F088
:100D00007D0900007D090000590D0000530D000011
:100D10006F49724B80220D2008701A70A2077FF570
:100D20002FAF26E740F20232904240F0ED81AA88D0
:100D300002F07F02042A69D86D88002D66D16449CB
:100D4000CDF804E0920011440A7842F002020A70E1
:100D5000C1E101238B5511E600238B550EE6B0F55A
:100D6000086F53D16349644A097811707146ED8860
:100D70008D4280F0E88252480478402DAE4644F01F
:100D8000020C28BF4FF0400E02EB0E0309EBCC0122
:100D9000029301234A604FEA0E48CEEB050101930E
:100DA0000025C82242EA080384F0010249F83C30D9
:100DB00035700270DFF814C1424BDFF8048149BB83
:100DC000BEF1400F7FF42DAF42F0020C09EBCC03D3
:100DD000029ADFF8F8E05A608DBB0D0445F08805F3
:100DE0009DF804304EF83C500A44337004701346AA
:100DF00040297FF416AF0021404A3B60118010E784
:100E0000AA8802F07F02042A40F28B81304A0F2325
:100E1000137006E74029D7D942F002020CEBC2005A
:100E2000029E4660BDB19DF8045035481D703346A2
:100E3000403988F8004040334CF83200DCE79DF838
:100E4000043033700D04029B047045F0C8050B4458
:100E50004EF83C50CCE79DF804501D70029B1D4895
:100E600088F80040403940334CF83200C4E719F0AC
:100E7000080F0CBF022303238B557FE521494A68E5
:100E8000002AC3D06C88B5F804E003E00C314A684E
:100E9000002ABBD00B88A342F8D14B887345F5D10B
:100EA000240A032C0CBF1178098960E7124A022139
:100EB000147054705BE700BF9420074001000400E9
:100EC0001C0DFF1FB00CFF1FB10CFF1F0000FF1F08
:100ED000C02007408800400088200740802007404D
:100EE00098200740600CFF1FB40CFF1F4C0CFF1F25
:100EF0001D0DFF1F280DFF1F200DFF1F5C0CFF1F86
:100F0000C8004000F82300008C200740B248116A56
:100F1000AC7804700C0600F19881D9F82820AF490C
:100F2000100600F1DB81D9F83020AC49120600F13F
:100F3000D081D9F83820A949130600F1C581D9F824
:100F40004020A649150600F1BA81D9F84820A349E6
:100F5000140600F1AF81D9F85020A049100600F125
:100F6000A481D9F858209D49120600F19981D9F839
:100F700060209A49130600F18E81D9F868209749BC
:100F8000150600F18381D9F870209449140600F108
:100F90007881D9F878209149100600F16D81D9F84F
:100FA00080208E49120600F16181D9F888208B4992
:100FB000130600F15581D9F890208849150600F1F3
:100FC0004981D9F898208549140600F1FF808448AA
:100FD000844A854901908548854D864C04970023B5
:100FE0000596029580460F4616461D4603943068C6
:100FF00028B1446800F056FA2046002CF9D10023AD
:101000003360029B38681A46002342F8253028B125
:10101000446800F047FA2046002CF9D100223A60DB
:10102000019A98F800301146002241F8042B039AE7
:101030000191023B4FF0000122F81510032B07D855
:10104000DFE803F05D025D024FF0010388F8003035
:101050000135042D06F1040607F1040708F1010823
:10106000C5D1654C654D2278654B049F059E0021D6
:10107000100729701A7000F19280624962780A7034
:101080000021C9F83010C9F838101107DFF84C8179
:101090006ED4A2785C49DFF844810A7000211207FF
:1010A000C9F85010C9F858104BD4E27857494B4C46
:1010B0000A7013074FF00001C9F87010C9F87810D2
:1010C00000F1AE8033780193002283F00105C9F866
:1010D0009020C9F898200021029188468E460A4641
:1010E0004B48047844F0020C09EBCC030393019BBA
:1010F000002B039B5A600CBF8822C82252E64FF097
:10110000000388F80030A3E7B0F5A06F7FF47EAE4F
:10111000012300250193DEE740F621229042F7D01B
:1011200074E66D88002D7FF471AE3A49CDF804E085
:10113000920011440A7822F002020A70CBE70221E1
:1011400015E600F08FF9002800F0EB800830324AF5
:10115000C8F86400C8F8602000F084F9002800F0A6
:10116000DA8008302D4AC9F86C00C9F868209CE77D
:1011700000F078F9002800F0E0800830264AC8F82E
:101180004400C8F8402000F06DF9002800F0CF803E
:101190000830224AC9F84C00C9F8482079E700F025
:1011A00061F9002800F0A58008301B4AC9F8240026
:1011B000C9F8202000F056F9002800F0948008308B
:1011C000164AC9F82C00C9F8282056E7D1F89C0027
:1011D000083800F067F9FAE6280DFF1F0000FF1F2E
:1011E000040DFF1FA00CFF1FF40CFF1F2C0DFF1F91
:1011F0004C0CFF1F5C10FF1FF42300001D0DFF1F90
:10120000C4200740C8200740CC200740D02007401A
:101210001C0DFF1FC020074088004000C800400090
:1012200000F020F9002870D008304F4AC4F884003C
:10123000C4F8802000F016F9002860D008304B4A2E
:10124000C9F88C00C9F888203CE7506A083800F0DB
:1012500029F962E6D1F89400083800F023F9B0E6E5
:10126000D1F88C00083800F01DF9A4E6D1F884000C
:10127000083800F017F998E6C86F083800F012F93E
:101280008DE6486F083800F00DF982E6C86E083820
:1012900000F008F977E6486E083800F003F96CE6CC
:1012A000C86D083800F0FEF861E6486D083800F0B7
:1012B000F9F856E6C86C083800F0F4F84BE6486CCC
:1012C000083800F0EFF840E6C86B083800F0EAF89C
:1012D00035E6486B083800F0E5F82AE6C86A0838B1
:1012E00000F0E0F81FE62A78C9F8280001322A70D9
:1012F000C3E62A78C9F8200001322A705AE72A7812
:10130000C9F8880001322A70DCE62A78C4F8800027
:1013100001322A708EE72A78C9F8680001322A70F3
:10132000C3E62A78C8F8600001322A7014E72A78E8
:10133000C9F8480001322A70ABE62A78C8F84000A4
:1013400001322A701FE740298E4628BF4FF0400E19
:1013500002EB0E0302930123CEEB01014FEA0E488C
:1013600000250193BCE600BF88004000C800400093
:101370002DE9F04100F034FD2F4C304B3048DFF8C0
:10138000D880304F304D314EDFF8D0C0DFF8D0E09C
:1013900000221A605A609A60DA601A615A619A6192
:1013A000DA611A625A629A62DA621A635A639A635B
:1013B000DA631A645A649A64DA641A655A659A653B
:1013C000DA651A665A669A66DA661A675A679A671B
:1013D000DA67C3F880202168C3F8842041F48021B3
:1013E0002160016841F040710160C3F3072188F872
:1013F000001004F52834C3F307411B0E3970CC34B8
:101400002B7000F12040FF238CF80030104D8EF837
:10141000003000F6041033700E49012308F8083C30
:10142000702622704FF40014102207F82C3C2E7006
:1014300004600A70BDE8F081348004400000FF1FA2
:1014400000D80040B0200740B420074010200740DB
:1014500035E400E0082107409C2007408020074039
:101460008820074072B60D480268B2FA82F30B2B4F
:1014700010DC4FF00041D94022EA0102026062B65E
:10148000074803EBC303DB00C2180021C15010461C
:101490005160704762B60020704700BFF806FF1F1A
:1014A0009803FF1F0D4B0E4AC31AA2FB03231B090F
:1014B0000B2B0CD80B4A127852B972B60A484FF06F
:1014C0000041026821FA03F31A43026062B67047D2
:1014D000064A1278002AF0D0FFF760B99803FF1F80
:1014E000398EE3381D0DFF1FF806FF1F280DFF1F63
:1014F00038B5164D2868E0B101884488A14213DD53
:1015000003191B7A83B104F10803C2180C1B0023D2
:1015100002E012F8011F21B10133A342F9D12046A4
:1015200038BD1C46204638BDFFF7BCFF00202860B0
:1015300038BD074B1B780BB9002038BD0220FFF7E0
:101540000FF928600028D7D1F6E700BF380DFF1F3C
:10155000280DFF1F0D4B1B78BBB910B50C4C216833
:1015600003F0FF024B883F2B07DC07330B4401F1EC
:10157000470003F8012F8342FBD140230B80012059
:10158000FFF770F90023236010BD7047300DFF1F77
:10159000340DFF1F08B5FEF769FFFEF76BFF00F083
:1015A00001F8FAE738B52C4C237803B138BD012394
:1015B0002370FFF79DFF002842D100F0F5F80028C6
:1015C0003BD100F087F9002834D100F019FA70BB44
:1015D00000F092FA40BB00F00BFB10BB00F084FB64
:1015E000E0B900232370EFF30583002BDED1EFF386
:1015F000108172B6194B186828B3194C227812BBA7
:1016000045691D60012323700DB3AA6101B962B65B
:1016100000254577836898472570C7E700F022FDCD
:10162000DFE700F01DFDD9E700F018FDD3E700F07B
:1016300013FDCDE700F00EFDC7E700F009FDC0E7A0
:1016400000F012FDB9E70029B0D162B638BD054BF4
:101650001D600029DCD1DAE73D0DFF1F5010FF1F90
:101660005410FF1F4C10FF1F30B42948294A2A4B41
:101670002A4D6024E121047011701B78284C082B3E
:1016800030D00A2B2748284937D00C2B0CBF3522E5
:101690003D2212232A60236002600B60234B244901
:1016A0001B78244ABBB101230B601360224B2349F2
:1016B0001B78234A012B26D9042B0FD9082B1ED9BE
:1016C000102B94BF862387230B6013601D4B0122D0
:1016D0001A7030BC70470B601360E7E784230B601F
:1016E0001360F3E700F58E200F4908300122132321
:1016F0002A60236002600B60D0E73922F7E7852378
:101700000B601360E2E780230B601360DEE700BF2D
:101710000040074001400740FC06FF1F08B003409F
:101720000CB0034008B00B400CB00B403F0DFF1F46
:1017300020B0034020B00B40FD06FF1F24B0034043
:1017400024B00B403E0DFF1F08B5104C08E0236885
:1017500059050DD423681A050FD42368DB0411D46E
:1017600023685803F3D5FFF7BFF823685905F1D56F
:1017700000F02AF823681A05EFD500F0BBF82368BB
:10178000DB04EDD500F04CF9EAE700BF34800440FB
:1017900008B5FFF7D9FF00BF014B10221A80704730
:1017A00000200540704700BF054A064B10781B78A3
:1017B000C0B2DBB2984238BF4030C01A704700BF99
:1017C000440DFF1F450DFF1FF0B4384B1A7912F07E
:1017D000300F2CD072B6997D01F0FF0200293DD068
:1017E00062B6334F334938780D78334E1C46C0B259
:1017F000EDB2431C402BE17928BF0023AB4202F13C
:10180000FF32C9B21CBFF154184612F0FF02F0D1EA
:101810002A4B1B68C2B23A704BB1A84236BFC5F121
:101820004005401B40192728C4BF01221A701F49D8
:10183000CA78D2B2150616D452060DD51B4B1B79A9
:101840005B0609D51E4B1F491B6800220A7003B1B5
:101850001A70164B3C22DA70F0BC70474022D979DE
:101860005A7462B6E3E70B791C06E5D5164B174EA2
:101870001C783378E4B2DBB29C420ED0144D01E008
:10188000A3420AD00133402B28BF00230879E85C2B
:10189000C0B2C871087D0728F2D9DBB203493370A2
:1018A0000B79180644BF7C23CB70C5E700A0064027
:1018B000440DFF1F450DFF1F880DFF1F400DFF1F2B
:1018C000CC0DFF1FC80DFF1FD00DFF1FC90DFF1F3F
:1018D000480DFF1F054A064B10781B78C0B2DBB2DB
:1018E000984238BF4030C01A704700BF440EFF1FF7
:1018F000D90DFF1FF0B4384B1A7912F0300F2CD0ED
:1019000072B6997D01F0FF0200293DD062B6334FD7
:10191000334938780D78334E1C46C0B2EDB2431CC3
:10192000402BE17928BF0023AB4202F1FF32C9B25C
:101930001CBFF154184612F0FF02F0D12A4B1B686D
:10194000C2B23A704BB1A84236BFC5F14005401B48
:1019500040192728C4BF01221A701F49CA78D2B281
:10196000150616D452060DD51B4B1B795B0609D5FF
:101970001E4B1F491B6800220A7003B11A70164BD8
:101980003C22DA70F0BC70474022D9795A7462B6B2
:10199000E3E70B791C06E5D5164B174E1C78337818
:1019A000E4B2DBB29C420ED0144D01E0A3420AD057
:1019B0000133282B28BF00230879E85CC0B2C87126
:1019C000087D0728F2D9DBB2034933700B7918067A
:1019D00044BF7C23CB70C5E700B00640440EFF1F18
:1019E000D90DFF1F040EFF1FD40DFF1F480EFF1F50
:1019F000D80DFF1F4C0EFF1F450EFF1FDC0DFF1FF4
:101A0000054A064B10781B78C0B2DBB2984238BF4B
:101A10004030C01A704700BF540EFF1F550EFF1F05
:101A200030B42B4B1A7994061FD52A48DA790378FB
:101A3000294901333F2B0978C8BF00238B42D2B21A
:101A400003D0264CD9B2E2540170254A116861B125
:101A5000244A1278D2B2934236BFC2F140029B1A96
:101A60009B18272BC4BF01230B70194AD378DBB214
:101A7000180611D45A060DD5154B1B795B0609D5EE
:101A8000194B1A491B6800220A7003B11A70104BD7
:101A90002C22DA7030BC704711790906EAD5144956
:101AA00010480C780178C9B28C420DD04A1C272A04
:101AB00084BF00210A460F4D054C98BFD1B2AA5CE5
:101AC000D2B2E2710170D5E76C21D170D2E700BFCC
:101AD00000C00640540EFF1F550EFF1F800EFF1F53
:101AE000500EFF1FC10EFF1FC40EFF1FC00EFF1FB1
:101AF000C80EFF1F580EFF1F054A064B10781B78B3
:101B0000C0B2DBB2984238BF4030C01A704700BF45
:101B1000D00EFF1FD10EFF1F30B42B4B1A79940645
:101B20001FD52A48DA790378294901333F2B0978F0
:101B3000C8BF00238B42D2B203D0264CD9B2E254A4
:101B40000170254A116861B1244A1278D2B29342D9
:101B500036BFC2F140029B1A9B18272BC4BF01233A
:101B60000B70194AD378DBB2180611D45A060DD57A
:101B7000154B1B795B0609D5194B1A491B680022C6
:101B80000A7003B11A70104B2C22DA7030BC704707
:101B900011790906EAD5144910480C780178C9B2C0
:101BA0008C420DD04A1C272A84BF00210A460F4DC3
:101BB000054C98BFD1B2AA5CD2B2E2710170D5E7F0
:101BC0006C21D170D2E700BF00D00640D00EFF1FBD
:101BD000D10EFF1FFC0EFF1FCC0EFF1F3D0FFF1F7E
:101BE000400FFF1F3C0FFF1F440FFF1FD40EFF1FAE
:101BF000054A064B10781B78C0B2DBB2984238BF5A
:101C00004030C01A704700BF4C0FFF1F4D0FFF1F21
:101C100030B42B4B1A7994061FD52A48DA79037809
:101C2000294901333F2B0978C8BF00238B42D2B228
:101C300003D0264CD9B2E2540170254A116861B133
:101C4000244A1278D2B2934236BFC2F140029B1AA4
:101C50009B18272BC4BF01230B70194AD378DBB222
:101C6000180611D45A060DD5154B1B795B0609D5FC
:101C7000194B1A491B6800220A7003B11A70104BE5
:101C80002C22DA7030BC704711790906EAD5144964
:101C900010480C780178C9B28C420DD04A1C272A12
:101CA00084BF00210A460F4D054C98BFD1B2AA5CF3
:101CB000D2B2E2710170D5E76C21D170D2E700BFDA
:101CC00000A00E404C0FFF1F4D0FFF1F780FFF1F8E
:101CD000480FFF1FB90FFF1FBC0FFF1FB80FFF1FDB
:101CE000C00FFF1F500FFF1F054A064B10781B78CF
:101CF000C0B2DBB2984238BF4030C01A704700BF54
:101D0000C80FFF1FC90FFF1F30B42B4B1A79940661
:101D10001FD52A48DA790378294901333F2B0978FE
:101D2000C8BF00238B42D2B203D0264CD9B2E254B2
:101D30000170254A116861B1244A1278D2B29342E7
:101D400036BFC2F140029B1A9B18272BC4BF012348
:101D50000B70194AD378DBB2180611D45A060DD588
:101D6000154B1B795B0609D5194B1A491B680022D4
:101D70000A7003B11A70104B2C22DA7030BC704715
:101D800011790906EAD5144910480C780178C9B2CE
:101D90008C420DD04A1C272A84BF00210A460F4DD1
:101DA000054C98BFD1B2AA5CD2B2E2710170D5E7FE
:101DB0006C21D170D2E700BF00B00E40C80FFF1FEA
:101DC000C90FFF1FF40FFF1FC40FFF1F3510FF1FA8
:101DD0003810FF1F3410FF1F3C10FF1FCC0FFF1FD8
:101DE00072B6184A184B19491160702280211A7076
:101DF0001A46197013781B06FCD510B5144B84B025
:101E0000186862B6134B144C984298BF00EB8000E0
:101E100001A998BF40000A2200F028F901A9204634
:101E2000002311F8012B01333AB10A2B20F8022FBD
:101E3000F7D11623237004B010BD5B00DBB2237012
:101E400004B010BD04000240000002400000074141
:101E50000C0002407F969800E407FF1F10B4EFF3D8
:101E6000108272B6437F33B9017F012908D003295C
:101E700010D00123437702B962B65DF8044B704776
:101E8000114C2168A1B1114943610B68836108605D
:101E90005861EEE70E4C216881B10E4943610B6831
:101EA0008361086058610C4B4FF080511960E0E786
:101EB000064B4161816120601860DAE7054B4161A2
:101EC000816120601860EEE75010FF1F4C10FF1F6B
:101ED0004010FF1F4410FF1F04ED00E010B4047F0A
:101EE0004160022CC26003D05DF8044BFFF7B6BF1F
:101EF00083685DF8044B184770B5EFF3108272B633
:101F00000C4C206880B10C4E00254369236073B1EE
:101F10009D6102B962B6457783689847EFF31082F6
:101F200072B620680028F0D102B962B670BD336085
:101F3000EFE700BF4010FF1F4410FF1FFFF7DCBF9B
:101F4000184A30B41468002C27D0036821688B42EB
:101F50000ED2CB1A00218460C1602360E060106063
:101F60000223037530BC704711688B42144608D3B6
:101F7000A2685B1A0360002AF6D18260C460A06088
:101F8000EEE7D268C2608460E060C568CB1A0222C6
:101F9000A8602360027530BC70478460C460106024
:101FA000DEE700BF4810FF1FF8B5224E34682CB39F
:101FB0002368002B3AD1204F1D4604E03468ECB171
:101FC0002368002B32D1A36803B1DD602069336040
:101FD000036825751B68BB4221D1037F4560022B36
:101FE000C46020D0FFF73AFF6368002BE6D023607F
:101FF0002046FFF7A5FF3468002CE1D1EFF31083F2
:1020000072B60E4A00211068116003B962B628B199
:102010008468FFF795FF20460028F9D1F8BD2246D5
:1020200000219847E0E783689847DDE7013B23609C
:10203000E4E700BF4810FF1FDD1E00005810FF1F1F
:10204000024A136801331360FFF7AEBF440CFF1F51
:10205000704700BF704700BF704700BF704700BFA8
:10206000704700BF704700BF704700BFF0B44D1EFF
:102070002E46002400E00134B0FBF2F302FB130013
:10208000092800F130078ABF3730F8B2C0B206F82D
:10209000010F1846002BEED10A1953704CB110787D
:1020A00015F8016F28700133E01A834202F80169C4
:1020B000F5DB0846F0BC704770B50F4E0F4D761B30
:1020C000B61018BF002405D0013455F8043B9847DA
:1020D000A642F9D10A4E0B4D761B00F0D1F9B6108D
:1020E00018BF002406D0013455F8043B9847A64297
:1020F000F9D170BD70BD00BF8C2400008C2400009D
:10210000942400008C240000024B13B1024800F01C
:1021100005B8704700000000292100000023014697
:102120001A46184600F014B838B5074D074C2C1B5A
:10213000A41005D0013C55F8043D9847002CF9D176
:10214000BDE8384000F0A6B9000000000000000023
:102150002DE9F047254C2568D5F8484106468846C4
:1021600092469946C4B360681F2817DC431C76B1B9
:1021700004EB80050122C5F888A0D4F888118240BC
:102180001143022EC4F88811C5F808911ED0023000
:10219000636044F820800020BDE8F087144B03B34F
:1021A0004FF4C870AFF300800446D0B1D5F8483181
:1021B000002780E88800C5F8484138460123C4F864
:1021C0008871C4F88C71002EE1D0D1E7D4F88C115D
:1021D0000A43C4F88C21DAE705F5A674C5F848412E
:1021E000C1E74FF0FF30BDE8F08700BF7C2400005E
:1021F000000000004008FE4340A004404408FE43A5
:1022000044A004400018FE4300C004403000FE43D8
:10221000309004403400FE43349004401C18FE43C8
:102220001CC004401018FE4310C004400818FE43B0
:1022300008C004400C18FE430CC004400C10FE43C0
:102240000CB004401010FE4310B004401810FE43C0
:1022500018B004401C10FE431CB004401410FE4390
:1022600014B004400418FE4304C004400010FE43B0
:1022700000B004400008FE4300A004400408FE43F0
:1022800004A004400C08FE430CA004400808FE43D0
:1022900008A004401418FE4314C004401818FE435C
:1022A00018C004400410FE4304B004400810FE436C
:1022B00008B004406820FE4368D004401400FE4388
:1022C000149004403800FE43389004403C00FE4324
:1022D0003C9004404000FE43409004404808FE43C8
:1022E00048A004404C08FE434CA004402808FE438C
:1022F00028A004402C08FE432CA004406020FE438C
:1023000060D004406420FE4364D004402010FE43AB
:1023100020B004402410FE4324B004402810FE43A3
:1023200028B004402C10FE432CB004404400FE436F
:10233000449004407000FE43709004407400FE43DB
:10234000749004406800FE43689004405008FE43C7
:1023500050A004405808FE4358A004405C08FE43C7
:102360005CA004405408FE4354A004402018FE43DF
:1023700020C004402418FE4324C004401008FE433B
:1023800010A004401408FE4314A004403818FE4373
:1023900038C004403418FE4334C004403018FE43B3
:1023A00030C004403C18FE433CC004402C18FE439F
:1023B0002CC004402820FE4328D004402C20FE439B
:1023C0002CD004400020FE4300D004400420FE43F3
:1023D00004D004400820FE4308D004400C20FE43F3
:1023E0000CD004401020FE4310D004401420FE43C3
:1023F00014D0044015191519000100000007FF1F33
:1024000012000000000200002C07FF1F490000001E
:10241000002201007807FF1F2100000000210100B9
:102420005E07FF1F09000000002200009C07FF1F3D
:102430001C000000002100003E07FF1F09000000F3
:1024400000030000E007FF1F000000000103090473
:102450001407FF1F0000000002030904B807FF1F54
:102460000000000003030904E407FF1F0000000050
:102470000000000000000000000000000008FF1F36
:10248000F8B500BFF8BC08BC9E46704709210000A3
:04249000350400000F
:04249400F8B500BFD8
:10249800FFFFFFFF0A0400001201100100000040C6
:1024A800C0168604760201020301000018035400D6
:1024B800650065006E0073007900640075006900AE
:1024C8006E006F0009024900020100C032090400D1
:1024D800000203000000092111010001221C00076D
:1024E80005830340000107050403400001090401B6
:1024F8000002030000000921110100012221000748
:1025080005810340000107050203200002000000C6
:1025180006C9FF0904A15C7508150026FF0095404F
:102528000975810295200976910295040976B10210
:10253800C000000006ABFF0A0002A10175081500E3
:1025480026FF00954009018102954009029102C0C9
:1025580026035400650065006E007300790064006E
:10256800750069006E006F0020005200610077005E
:102578004800490044000000040309040C0300005B
:102588000000000000000000000000000000000043
:10259800000000000000000000000000EC0AFF1F1F
:1025A800540BFF1FBC0BFF1F0000000000000000C1
:1025B8000000000000000000000000000000000013
:1025C8000000000000000000000000000000000003
:1025D80000000000000000000000000000000000F3
:1025E80000000000000000000000000000000000E3
:1025F80000000000000000000000000000000000D3
:1026080000000000000000000000000000000000C2
:1026180000000000000000000000000000000000B2
:1026280000000000000000000000000000000000A2
:102638000000000000000000000000000000000092
:1026480001000000000000000E33CDAB34126DE62F
:10265800ECDE05000B000000000000000000000098
:102668000000000000000000000000000000000062
:102678000000000000000000000000000000000052
:102688000000000000000000000000000000000042
:102698000000000000000000000000000000000032
:00000001FF
